:100000000C9468000C9417040C94D6010C94D20044
:100010000C94D2000C94D2000C94D2000C94D20018
:100020000C94D2000C94D2000C94D2000C94D20008
:100030000C94D2000C94D2000C94D2000C94D200F8
:100040000C94D2000C94D2000C94D2000C947E0438
:100050000C94D2000C94AD040C94D2000C94D200F9
:100060000C94D2000C94D2000C94D2000C94D200C8
:100070001B5B373B3148001B5B304B001B5B363B47
:100080003148001B5B324A1B5B480D0A496E69749C
:100090000D0A00557000446F776E004C6566740061
:1000A00052696768740043656E746572004E6F6EC6
:1000B0006500930096009B00A000A600AD001B5BAE
:1000C000373B3148001B5B353B31481B5B304B00F5
:1000D00000E805BF00E200BF4FEFF0E1E0E00FEF06
:1000E0001EE03FEF2FEF208321913223003019F0E3
:1000F00001190C947200103021F011190FEF0C94BB
:1001000072003F3F09F04E7FF0E1E0E00FEF1EE0AC
:1001100038E828E8208321913223003019F00119B2
:100120000C948900103021F011190FEF0C94890004
:10013000383809F04D7FF0E1E0E00FEF1EE030E0ED
:1001400020E0208321913223003019F001190C9412
:10015000A000103021F011190FEF0C94A0003030E6
:1001600009F04B7FF1E1E0E0408311241FBECFEFA7
:10017000D4E0DEBFCDBF10E1A0E0B0E1E8E5F3E1FF
:1001800002C005900D92AC33B107D9F710E1ACE392
:10019000B0E101C01D92AD3CB107E1F70E94D4006F
:1001A0000C94AA090C9400002F923F924F925F92F8
:1001B0006F927F928F929F92AF92BF92CF92DF9277
:1001C000EF92FF920F931F93DF93CF93CDB7DEB7DC
:1001D00060970FB6F894DEBF0FBECDBF109100112F
:1001E000F8940E940E050E9426040E944102789411
:1001F00080915F10909160109093CA108093C91005
:1002000083E890E09F938F930E94B306DE011896D7
:10021000E3E2F0E189E001900D928150E1F768E0BE
:1002200070E0CE0108960E94B601812F90E09F9366
:100230008F9380E090E19F938F930E949E06329A65
:1002400000E010E0EE24FF248DB79EB706960FB6AF
:10025000F8949EBF0FBE8DBF6E010894C11CD11CC7
:100260004CE7242E40E0342E37E7432E30E0532E67
:1002700027E1622E20E1722E90E7892E90E0992EE0
:100280008CECA82E84E0B82E80913C108823E1F0FD
:100290000894E11CF11CFF92EF9283E190E19F939F
:1002A0008F93DF92CF920E94DA0667E070E0C6017A
:1002B0000E94B60110923C108DB79EB706960FB6FD
:1002C000F8949EBF0FBE8DBF80914110882321F00E
:1002D0000E943203109241100F5F1F4F0A3F110519
:1002E00049F53F922F920E94B3065F924F920E946F
:1002F000B30681E00E949E018C0180E00E949E0175
:100300000F5710401F930F938F5790409F938F93D9
:100310007F926F920E949E069F928F920E94B306D8
:1003200000E010E08DB79EB70C960FB6F8949EBF14
:100330000FBE8DBFC5010197F1F7A6CF823018F02F
:1003400020E030E011C0E0912C10F0912D1090E0F1
:10035000880F991F80832899FECFE0912C10F0918F
:100360002D108081282F30E0C9010895AC01109232
:10037000421080914210882311F4C49805C08091E6
:100380004210813009F4C39820E030E00AC0FA013D
:10039000E20FF31F80818FB9779BFECF8FB12F5F64
:1003A0003F4F261737079CF3C49A08951F920F9268
:1003B0000FB60F9211248F9381E080933C108F91A0
:1003C0000F900FBE0F901F901895109242108091C1
:1003D0004210882311F4C49805C0809142108130E6
:1003E00009F4C3981FB8779BFECF8FB1282F30E058
:1003F00021503040309334102093331080914210BC
:10040000882311F4C49A05C080914210813009F408
:10041000C39A8FEF2F3F380799F12630310584F5C5
:1004200085EC90E09F938F930E94B306E091331088
:10043000F0913410EE0FFF1FEE54FF4F6591749151
:100440008091491090914A100E941F068091491096
:1004500090914A109F938F938EE290E19F938F9398
:100460000E949E068EEB90E09F938F930E94B306AE
:100470008DB79EB708960FB6F8949EBF0FBE8DBF7E
:1004800008958B9885B7886085BF8BB780688BBFD0
:1004900088E090E00E9420058093491090934A10D4
:1004A0000895982F80914210882311F4C49805C0B4
:1004B00080914210813009F4C39882E08FB9779B14
:1004C000FECF8FB19FB9779BFECF8FB16FB9779B6E
:1004D000FECF8FB180914210882311F4C49A089501
:1004E00080914210813009F4C39A0895982F809129
:1004F0004210882311F4C49805C0809142108130C5
:1005000009F4C39883E08FB9779BFECF8FB19FB971
:10051000779BFECF8FB11FB8779BFECF9FB18091A5
:100520004210882311F4C49A05C080914210813092
:1005300009F4C39A892F0895F894BB9AC39A85B792
:10054000826085BF8BB780648BBF81E0809342104F
:100550006FE18BE20E94510260E280E60E9451024C
:1005600060E48FE00E9451028FE00E94760290E0EA
:10057000803409F491E0892F0895DC0180914010C6
:10058000882309F46EC0F89481E080934210809132
:100590004210882311F4C49805C080914210813024
:1005A00009F4C39880E48FB9779BFECF8FB19C91FB
:1005B000892F8695869586958FB9779BFECF8FB1CB
:1005C00097709FB9779BFECF8FB11FB8779BFECFF7
:1005D0008FB11FB8779BFECF8FB1FD012281822F93
:1005E0008F708FB9779BFECF8FB190E030E02F7086
:1005F000307008C0EA0FFB1F83818FB9779BFECF55
:100600008FB19F5FE92FF0E0E217F3079CF3809131
:100610004210882311F4C49A05C0809142108130A1
:1006200009F4C39A80914210882311F4C49805C03C
:1006300080914210813009F4C39881E88FB9779B8B
:10064000FECF8FB180914210882311F4C49A05C067
:1006500080914210813009F4C39A81E08093401068
:100660007894089581E0809342108091421088230D
:1006700011F4C49805C080914210813009F4C398E8
:1006800083E08FB9779BFECF8FB18CE28FB9779BD8
:10069000FECF8FB11FB8779BFECF9FB120913E1048
:1006A00080914210882311F4C49A05C080914210B1
:1006B000813009F4C39A90933E1080913E108130AE
:1006C00039F585E60E9476028F7080933D10809107
:1006D0004210882311F4C49805C0809142108130E3
:1006E00009F4C39882E98FB9779BFECF8FB190E070
:1006F0000AC01FB8779BFECF8FB1E92FF0E0E55B12
:10070000FF4E80839F5F80913D10981790F32AC021
:1007100080913E10823091F585E70E9476028F70BD
:1007200080933D1080914210882311F4C49805C035
:1007300080914210813009F4C39886E98FB9779B84
:10074000FECF8FB190E00AC01FB8779BFECF8FB16C
:10075000E92FF0E0E55BFF4E80839F5F80913D10C5
:10076000981790F380914210882309F458C0809123
:100770004210813009F05AC0C39A0895922780919F
:100780003E10843059F580914210882311F4C498AA
:1007900005C080914210813009F4C39885E08FB97B
:1007A000779BFECF8FB18CE28FB9779BFECF8FB155
:1007B0009FB9779BFECF8FB11FB8779BFECF8FB1CC
:1007C00080914210882311F4C49A05C08091421090
:1007D000813009F4C39A109240100895809142101C
:1007E000882311F4C49805C080914210813009F427
:1007F000C39885E08FB9779BFECF8FB18CE28FB91C
:10080000779BFECF8FB19FB9779BFECF8FB11FB87B
:10081000779BFECF8FB180914210882311F4C49A48
:10082000089580914210813009F4C39A08951F926F
:100830000F920FB60F9211248F9381E08093411095
:100840008F910F900FBE0F901F901895C49A87B389
:10085000806B87BB81E58DB90895E0914310F091DD
:100860004410EE59FF4E80838091431090914410C4
:10087000019690934410809343108091431090917F
:100880004410C09721F410924410109243108091AC
:100890006110882361F4E0914510F0914610EE5903
:1008A000FF4E80818CB981E080936110559A80E081
:1008B00090E00895AC0180919210882319F420E013
:1008C00030E01AC01092921020E030E00AC0FA0125
:1008D000E20FF31FD901AD56BF4E8C9180832F5F7D
:1008E0003F4F8091471090914810281739077CF3AB
:1008F0001092481010924710C90108951F920F924C
:100900000FB60F9211248F939F93EF93FF93E09173
:100910004710F09148108CB1ED56FF4E8083E09166
:100920004710F0914810ED56FF4E80818D3019F43C
:1009300081E0809392108091471090914810019629
:100940009093481080934710FF91EF919F918F9162
:100950000F900FBE0F901F9018951F920F920FB619
:100960000F9211242F933F938F939F93EF93FF93B5
:100970008091451090914610019690934610809377
:1009800045108091451090914610C09721F4109227
:1009900046101092451020914510309146108091DC
:1009A0004310909144102817390749F0E091451001
:1009B000F0914610EE59FF4E80818CB903C05598D6
:1009C00010926110FF91EF919F918F913F912F9124
:1009D0000F900FBE0F901F901895EF92FF920F93FC
:1009E0001F93CF93DF937C018B01C0E0D0E00CC05C
:1009F0006091C9107091CA10F701EC0FFD1F808142
:100A000090E00E9472062196C017D1078CF3DF9107
:100A1000CF911F910F91FF90EF90089510BC8FE040
:100A200089B988E98AB986E880BD60E070E08DE226
:100A300094E00E9426069093601080935F100895C2
:100A4000CF93DF93BC018230910510F462E070E037
:100A5000A091C510B091C610ED0140E050E0E0E07B
:100A6000F0E021C0888199818617970769F48A810F
:100A70009B81309719F09383828304C09093C610B2
:100A80008093C510FE0133C06817790738F441150B
:100A9000510519F08417950708F4AC01FE018A810D
:100AA0009B819C01E9012097E9F641155105A1F1CF
:100AB000CA01861B970B049708F4BA01E0E0F0E046
:100AC00029C08D919C91119784179507F1F46417B3
:100AD000750779F4ED018A819B81309719F0938332
:100AE000828304C09093C6108093C510FD01329696
:100AF0004CC0CA01861B970BFD01E80FF91F6193DB
:100B0000719302978D939C9340C0FD0182819381E4
:100B10009C01D9011097A9F68091C3109091C4103F
:100B2000892B41F480913710909138109093C41024
:100B30008093C3104091391050913A1041155105DE
:100B400041F44DB75EB78091351090913610481B37
:100B5000590B2091C3103091C410CA01821B930B12
:100B60008617970780F0AB014E5F5F4F841795079C
:100B700050F0420F531F5093C4104093C310F9011B
:100B80006193719302C0E0E0F0E0CF01DF91CF917B
:100B90000895CF93DF93009709F44EC0EC0122979C
:100BA0001B821A82A091C510B091C610109701F156
:100BB00040E050E0AC17BD0700F1BB83AA83FE0103
:100BC00021913191E20FF31FAE17BF0771F48D91A0
:100BD0009C911197280F391F2E5F3F4F398328832F
:100BE000FD01828193819B838A834115510569F4BC
:100BF000D093C610C093C5101FC0FD0182819381A0
:100C0000AD01009711F0DC01D5CFFA01D383C28387
:100C100021913191E20FF31FCE17DF0769F488812C
:100C20009981280F391F2E5F3F4FFA0131832083AE
:100C30008A819B8193838283DF91CF910895FB0109
:100C4000DC0105900D920020E1F708950F931F93AA
:100C5000CF93DF938C01EB01009731F4611571059F
:100C600019F420E030E038C06EE070E081E090E000
:100C70000E94DC08FC019C01009771F180E88383ED
:100C8000209771F0D387C28781E883838091C71052
:100C90009091C810892B21F4F093C810E093C710ED
:100CA00001151105C9F01187008783818260838354
:100CB0008091C9109091CA10892B71F4F093CA10D9
:100CC000E093C9108091CB109091CC10892B21F426
:100CD000F093CC10E093CB10C901DF91CF911F911D
:100CE0000F9108950F931F93CF93DF938C01EB0126
:100CF0008B8181FF1BC082FF0DC02E813F818C81C3
:100D00009D812817390764F4E881F9810193F983FB
:100D1000E88306C0E885F985802F0995892B31F491
:100D20008E819F8101969F838E8302C00FEF1FEFFC
:100D3000C801DF91CF911F910F910895A0E0B0E01D
:100D4000E4EAF6E00C948309FE0135966191719115
:100D5000AF018091C9109091CA100E94FD062096A3
:100D6000E2E00C949F09A0E0B0E0E9EBF6E00C941F
:100D700083099E012B5F3F4FF901619171919F01A2
:100D8000A091C910B091CA10FD018381886083834E
:100D9000A9018091C9109091CA100E94FD06E091AE
:100DA000C910F091CA102381277F23832096E2E0A7
:100DB0000C949F09AEE0B0E0E0EEF6E00C948109FF
:100DC0000D891E8986E08C831A8309838FEF9FE744
:100DD0009E838D83CE014996AC016F89788DCE01BB
:100DE00001960E94FD062F813885020F131FF8011E
:100DF00010822E96E4E00C949D09ABE0B0E0E3E0B5
:100E0000F7E00C9473093C012B015A01FC01178295
:100E10001682838181FD03C06FEF7FEFC8C19AE026
:100E2000892E1E010894211C311CF3012381F2013B
:100E300023FD859123FF81912F01882309F4B4C1FB
:100E4000853239F423FD859123FF81912F0185326D
:100E500029F4B30190E00E947206E7CF982FDD24B9
:100E6000CC249924FFE1FD15D0F09B3269F09C322F
:100E700028F4903259F0933291F40EC09D3249F02B
:100E8000903369F441E024C052E0D52A84E0D82AA6
:100E900028C098E0D92A25C0E0E1DE2A22C0D7FC8C
:100EA00029C0892F80538A3070F4D6FE05C0989CE3
:100EB000902C1124980E15C0C89CC02C1124C80E6B
:100EC000F0E2DF2A0EC09E3229F4D6FC6DC140E468
:100ED000D42A07C09C3619F450E8D52A02C09836A7
:100EE00049F4F20123FD959123FF91912F0199235C
:100EF00009F0B8CF892F8554833018F080528330A1
:100F000038F444E050E0A40EB51E5FE359830FC0EF
:100F1000933631F0933779F0933509F056C020C0FD
:100F2000F5018081898342E050E0A40EB51E710175
:100F300001E010E012C0F501E080F180D6FC03C0B2
:100F40006FEF7FEF02C0692D70E042E050E0A40E29
:100F5000B51EC7010E940A098C015FE7D52214C0A3
:100F6000F501E080F180D6FC03C06FEF7FEF02C097
:100F7000692D70E042E050E0A40EB51EC7010E944A
:100F8000F8088C0150E8D52AD3FE07C01AC0B30177
:100F900080E290E00E947206CA948C2D90E00817BF
:100FA0001907A8F30EC0F701D7FC8591D7FE8191F0
:100FB0007F01B30190E00E947206C110CA940150F3
:100FC00010400115110579F7ECC0943611F09936EF
:100FD00071F5D7FE08C0F501E080F1800281138130
:100FE00044E050E00AC0F501808191817C01002736
:100FF000F7FC0095102F42E050E0A40EB51E5FE60E
:10100000D52217FF0AC010950095F094E094E11CDA
:10101000F11C011D111D80E8D82A2AE030E0A10151
:10102000C801B7010E941509F82EF21840C0953783
:1010300029F41D2D1F7E2AE030E01DC01D2D197FD3
:101040009F3661F0903720F4983509F0ADC00FC09D
:10105000903739F0983709F0A7C004C028E030E095
:101060000AC0106114FD146020E130E004C014FDDA
:10107000166020E132E017FF08C0F5016081718140
:101080008281938144E050E008C0F5018081918124
:10109000BC0180E090E042E050E0A40EB51EA1014A
:1010A0000E941509F82EF2188FE7D82ED122D6FE0D
:1010B0000BC05EEFD522F91438F4D4FE07C0D2FC81
:1010C00005C08FEED82202C01F2D01C0192DD4FEFD
:1010D0000DC0FE01EF0DF11D8081803319F499EEF2
:1010E000D92208C01F5FD2FE05C003C08D2D8678AF
:1010F00009F01F5F0D2DD3FC14C0D0FE0FC01C15CE
:1011000010F09F2C0BC09F2C9C0C911A1C2D06C01C
:10111000B30180E290E00E9472061F5F1C15C0F3CD
:1011200004C01C1510F4C11A01C0CC2404FF10C067
:10113000B30180E390E00E94720602FF1EC001FD31
:1011400003C088E790E002C088E590E0B3010CC0DE
:10115000802F867891F001FF02C08BE201C080E20F
:10116000D7FC8DE2B30190E00E94720606C0B30185
:1011700080E390E00E9472069A94F914C0F3FA9406
:10118000F101EF0DF11DB301808190E00E94720624
:10119000FF20A9F706C0B30180E290E00E9472062A
:1011A000CA94CC20C1F741CEF30166817781CB018F
:1011B0002B96E2E10C948F090F931F93CF93DF934B
:1011C000689F8001699F100D789F100D1124C80140
:1011D0000E942005EC01009729F0A80160E070E072
:1011E0000E940309CE01DF91CF911F910F910895C5
:1011F000FC010590615070400110D8F780959095E2
:101200008E0F9F1F0895DC0101C06D934150504027
:10121000E0F70895FC016150704001900110D8F78B
:10122000809590958E0F9F1F0895FA01AA27283068
:1012300051F1203181F1E8946F936E7F6E5F7F4FA3
:101240008F4F9F4FAF4FB1E03ED0B4E03CD0670F1F
:10125000781F891F9A1FA11D680F791F8A1F911D72
:10126000A11D6A0F711D811D911DA11D20D009F4C2
:1012700068943F912AE0269F11243019305D319304
:10128000DEF6CF010895462F4770405D4193B3E0ED
:101290000FD0C9F7F6CF462F4F70405D4A3318F094
:1012A000495D31FD4052419302D0A9F7EACFB4E045
:1012B000A6959795879577956795BA95C9F70097FD
:1012C0006105710508959B01AC010A2E069457959E
:1012D000479537952795BA95C9F7620F731F841FF5
:1012E000951FA01D08952F923F924F925F926F928B
:1012F0007F928F929F92AF92BF92CF92DF92EF92A6
:10130000FF920F931F93CF93DF93CDB7DEB7CA1B26
:10131000DB0B0FB6F894DEBF0FBECDBF09942A8851
:10132000398848885F846E847D848C849B84AA84F9
:10133000B984C884DF80EE80FD800C811B81AA8186
:10134000B981CE0FD11D0FB6F894DEBF0FBECDBF51
:08135000ED010895F894FFCFB0
:101358004D656D7465737420726573756C743A208D
:1013680025780025640A00583A20256420593A2037
:101378002564004279676765726E0A00FF1F25734E
:0C1388000D0A0005002000CD10FF1E0023
:00000001FF
